:0200000480007A
:100000006F00000B1300000013000000130000003D
:100010001300000013000000130000001300000094
:10002000232E11FE232C51FE232A61FE232871FE6C
:100030002326A1FE2324B1FE2322C1FE2320D1FECC
:10004000232EE1FC232CF1FC232A01FD232811FDA2
:100050002326C1FD2324D1FD2322E1FD2320F1FD30
:10006000130101FCEF00400B8320C10383228103B5
:1000700003234103832301030325C1028325810256
:1000800003264102832601020327C1018327810140
:100090000328410183280101032EC100832E810022
:1000A000032F4100832F010013010104730020304E
:1000B00097410000938101031771000013018185AE
:1000C0001385C18197650000938505446308B500D9
:1000D00023200500130545006FF05FFF1745000062
:1000E000130505801301C1FF973500009385457FF7
:1000F000630EB50083260500130545002320A100EB
:10010000E7800600032501006FF01FFE1301410088
:08011000EF20107F6F000000DA
:100118006780000003C75183930710046304F70046
:10012800678000008327050003A7C1839387970092
:10013800B387E7402320F5006780000003A64184C9
:1001480063080600032706002320E50003A6418470
:1001580083A5C1831306C6001305A0006F00D00F46
:10016800130101FF2320210183A741842324810057
:100178000324050003A707002322910083AE47004C
:1001880003AE870003A3070183A8470103A88701DB
:1001980083A5070203A6470283A687022326110028
:1001A8009304050003A5C70183A7C7022320E40021
:1001B80003A70400232EA4002326F4022322D4013B
:1001C800930750002324C40123286400232A140120
:1001D800232C04012320B4022322C4022324D402A2
:1001E80023A6F4002326F4002320E40013050400CA
:1001F800EFF0DFF4832744006380070883A7040037
:100208008320C1000324810083AF070003AF4700A8
:1002180083AE870003AEC70003A3070183A8470185
:1002280003A8870183A5C70103A6070283A647027F
:1002380003A7870283A7C70223A0F40123A2E4012E
:1002480023A4D40123A6C40123A8640023AA14016B
:1002580023AC040123AEB40023A0C40223A2D40219
:1002680023A4E40223A6F402032901008324410005
:10027800130101016780000003A584009307600053
:10028800930584002326F400EF00D01083A741844F
:100298000325C4001306C40083A707008320C100F8
:1002A800832441002320F400032481000329010052
:1002B8009305A000130101016F00007A83C75183E1
:1002C80083A681839387F7FB93B71700B3E7D7001B
:1002D80023ACF18213072004238AE182678000009F
:1002E80013071004A38AE18223AC0182678000000F
:1002F800130101F613050003232E1108232C81088E
:10030800232C81072326B107232A910823282109B2
:100318002326310923244109232251092320610975
:10032800232E7107232A91072328A107EF00501FC6
:1003380023A0A18413050003EF00901E83A7018466
:1003480023A2A1842320F500930720002324F5008D
:10035800B7350080930780022326F5001306F001C5
:10036800938545122322050013050501EF00D034BB
:10037800373700809307C768032EC76803A3470071
:1003880083A8870003A8C70083A5070103A6470120
:1003980083A6870103D7C70183C7E701B74D00804C
:1003A800231EE102230FF10213874D9F9307A0003C
:1003B8001305A000232EF7642320C1032322610222
:1003C80023241103232601032328B102232AC1026F
:1003D800232CD102EF00D02C3735008013054514AB
:1003E800EF00D0271305A000EF00902B83A701830F
:1003F800638007623735008013054517EF00102624
:100408001305A000EF00D029373500801305051D1E
:10041800EF0090131305A000EF00902837350080F7
:100428009305800C13058520EF001012EF001028AB
:10043800373400808327C46A373D0080832BCD6C16
:100448002324F10023A6A182930910001304C46A8F
:1004580093042000EFF0DFE8EFF05FE68347E40164
:1004680003264401032E4400032384008328C40088
:1004780003280401832684010357C401832E8100C5
:10048800230FF104930501049307100013050102DB
:10049800232AC104232EF100232A91002320D10509
:1004A8002322C105232461042326110523280105DD
:1004B800232CD104231EE104EF0000670326410129
:1004C8001335150023ACA18263CAC4029317260012
:1004D800B387C7009387D7FF13050600930530003D
:1004E80013068101232CF100EF0000570326410178
:1004F80013061600232AC100E3DAC4FC832681010F
:100508001385C18493854D9FEF00005603A5418450
:10051800930A1004130A3000EFF09FC403C7418305
:1005280093070004930CCD6C63F4E70213850A006B
:1005380093053004EF00405D8327C10113871A003B
:100548006302F54683C74183937AF70FE3F057FFB9
:100558008325410113050A0093891900EF2090278C
:10056800832A81012326A10093850A00EF20D02841
:10057800130A050013054101232A4101EFF09FB931
:100588009307900CE398F9ECEF00501223A4A18292
:100598003735008013058523EF00500C1305A000A4
:1005A800EF0010103735008013058524EF00100B7D
:1005B8001305A000EF00D00E83A5C1833735008056
:1005C8001305052837340080EF00007893055000A4
:1005D8001305C429EF00407783A581833735008050
:1005E8001305852BEF004076930510001305C429E9
:1005F800EF00807583C55183373500801305452D7D
:10060800EF008074B7340080930510041385042F1D
:10061800EF00807383C54183373500801305C530EB
:10062800EF008072930520041385042FEF00C0713A
:100638009387C18483A50702373500801305853267
:10064800EF008070930570001305C429EF00C06F98
:10065800B74700809387479F83A5C76537350080D4
:1006680013054534EF00406E373500801305053615
:10067800EF00C07E373500801305C538EF00007ED7
:1006880083A74184B73D008013858D3983A5070072
:10069800B73C0080B73B0080EF00006B3735008027
:1006A8001305453BEF00807B83A7418413854C3EAF
:1006B800373B008083A54700B73900803739008071
:1006C800EF008068930500001305C429EF00C06798
:1006D80083A7418413850B4083A58700EF00C0667C
:1006E800930520001305C429EF00006683A7418401
:1006F8001305CB4183A5C700EF00006593051001E2
:100708001305C429EF00406483A5418413858943F8
:1007180093850501EF00406313054945EF00007418
:100728003735008013058548EF00407383A701849F
:1007380013858D3983A50700EF00006137350080E8
:1007480013058549EF00807183A7018413854C3E0A
:1007580083A54700EF00405F930500001305C429F7
:10076800EF00805E83A7018413850B4083A5870073
:10077800EF00805D930510001305C429EF00C05CED
:1007880083A701841305CB4183A5C700EF00C05B95
:10079800930520011305C429EF00005B83A501849C
:1007A8001385894393850501EF00005A13054945D0
:1007B800EF00C06A83254101373500801305854D58
:1007C800EF008058930550001305C429EF00C05767
:1007D8008327C100373500801305454FB38A574139
:1007E80093973A00B38A5741B3854A41EF00C05501
:1007F8009305D0001305C429EF0000558325810116
:100808003735008013050551EF000054930570003B
:100818001305C429EF0040538325C10137350080F3
:100828001305C552EF004052930510001305C42963
:10083800EF00805137350080930501021305855478
:10084800EF0080503735008013054556EF000061F2
:10085800373500809305010413058559EF00C04E14
:10086800373500801305455BEF00405F1305A00096
:10087800EF00006303A7C18283A581829307301F1D
:10088800B385E54023A2B18263D0B71A373500801B
:1008980013050564EF00404B03A54182EF200037A4
:1008A80013040500EF20C048B747008003A6078E51
:1008B80083A6478EEF108007B747008003A6878E70
:1008C80083A6C78EEF009005EF20405723A0A18292
:1008D800B747008003A5078F93050400EF10007445
:1008E80023AEA1803735008013054565EF00C0456C
:1008F80003A54182EF208031B747008093050500AA
:1009080003A5478FEF10807113040500EF2000291D
:1009180093040500EF20802F9305050013050400BC
:10092800EF105060B747008083A5878FEF1090289D
:10093800EF20C02613040500373500809385040096
:1009480013054568EF0040409307900063D0871077
:10095800373500809305040013058568EF00C03E15
:100968001305A000EF00C0538320C10903248109A7
:1009780083244109032901098329C108032A81081D
:10098800832A4108032B0108832BC107032C810705
:10099800832C4107032D0107832DC1061301010A8A
:1009A800678000009305C10113050000EF00801E59
:1009B80003AE4C0003A38C0083A8CC0003A80C0151
:1009C80003A54C0183A58C0103D6CC0103C7EC0118
:1009D80083C74183938A1A00232071052322C10506
:1009E800232461042326110523280105232AA104B1
:1009F800232CB104231EC104230FE10423AE318349
:100A080093FAFA0F138A0900E3F257B36FF05FB451
:100A1800373500801305051AEF0040441305A00080
:100A2800EF0000486FF05F9E373500801305855E44
:100A3800EF00C0423735008013050562EF00004221
:100A48001305A000EF00C0456FF01FF21305000367
:100A5800EF0000456FF0DFEF13052500B305B50083
:100A68002320B60067800000130101FE2326310110
:100A780093095600232A910093942900232C81007E
:100A880023282101232E1100B30495001309060021
:100A98001384050023AC340723A0D40023A2D40078
:100AA800138509009305800CEF20C0521319290003
:100AB800B3072501B307F40003A7070123AA3701E9
:100AC80023AC37011307170023A8E70083A7040006
:100AD8003304A400330424013716000033048600CD
:100AE800232AF4FA8320C10103248101130750004B
:100AF80023AEE18283244101032901018329C10036
:100B080013010102678000001375F50F93F5F50FC7
:100B18006306B5001305000067800000A38AA18260
:100B28001305100067800000130101FF23248100D2
:100B38002322910023261100130405009384050045
:100B480083C5340003452400EFF01FFCE31A05FEBB
:100B58009385040013050400EF0080449307000008
:100B68006358A0001307A00023AEE182930710008A
:100B78008320C100032481008324410013850700DA
:100B880013010101678000001305E5FF1335150007
:100B980067800000130101FF2324810023229100B4
:100BA800232611001304050093840500EFF0DFFDF0
:100BB800630E050223A08400930710006300F40469
:100BC8006304040413072000630CE4049307400043
:100BD8006314F40023A0E4008320C10003248100EF
:100BE800832441001301010167800000930730004E
:100BF80023A0F40093071000E314F4FC03A7C183B7
:100C08009307400663DAE7028320C10003248100CA
:100C180023A0040083244100130101016780000020
:100C28008320C1000324810023A0F4008324410011
:100C380013010101678000008320C10003248100A3
:100C48009307300023A0F40083244100130101011D
:100C580067800000130101FF23248100232611006F
:100C68001304050003450500630A05001304140076
:100C7800EF00002303450400E31A05FE8320C100AA
:100C88000324810013010101678000006F004021E7
:100C9800130101FD2322910223261102232481023C
:100CA800232021039304050063440506130901006A
:100CB800130409006F004002EF20403C930705032E
:100CC80013041400138504009305A000A30FF4FE79
:100CD800EF208032930405009305A00013850400DB
:100CE800E39C04FCE30A24FD1304F4FF0345040019
:100CF800EFF0DFF9E31A24FF8320C1020324810205
:100D080083244102032901021301010367800000C3
:100D18001305D002EFF09FF7B30490406FF01FF96E
:100D280003A78184B307A7003765008023A4F18453
:100D380013054510930600403305E50063D4F6001B
:100D48007300100067800000130101FB232C410190
:100D58002326110223248102232291022320210326
:100D6800232E3101232A5101130A050003450500EA
:100D78002322F10493074103232AB102232CC10241
:100D8800232ED1022320E104232401052326110563
:100D98002326F1006308050213040000930A500299
:100DA800930430061309300793094006630E550370
:100DB800EFF0DFED13041400B3078A0003C5070042
:100DC800E31605FE8320C102032481028324410225
:100DD800032901028329C101032A8101832A4101D0
:100DE8001301010567800000930614003307DA0039
:100DF8006F000001638C270363863705938616000E
:100E0800834707001384060013071700E38407FAD3
:100E1800E39297FE8327C10003A507009387470045
:100E28002326F100EFF09FE66FF0DFF88327C1007B
:100E380003A50700938747002326F100EFF09FE101
:100E48006FF05FF78327C10003A50700938747006A
:100E58002326F100EFF0DFE36FF0DFF5130101FF68
:100E680023248100232611001304050003450500EF
:100E7800630A050013041400EF0080020345040010
:100E8800E31A05FE1305A000EF0080018320C100CE
:100E9800032481001305000013010101678000008D
:100EA800B70710F023A0A7F067800000B70710F07D
:100EB80003A507F167800000B3C7A50093F73700C3
:100EC8003307C500639607009307300063E4C70241
:100ED80093070500636CE5006780000083C6050082
:100EE8009387170093851500A38FD7FEE3E8E7FEE5
:100EF8006780000093773500639207089307050021
:100F08009376C7FF138606FE63F6C70883A305001A
:100F180083A2450083AF850003AFC50083AE0501FA
:100F280003AE450103A3850183A8C5019385450246
:100F38009387470203A8C5FF23AE77FC23A057FE7B
:100F480023A2F7FF23A4E7FF23A6D7FF23A8C7FF01
:100F580023AA67FE23AC17FF23AE07FF6FF0DFFA63
:100F680083C605009387170093851500A38FD7FEC6
:100F780093F63700E39606FE6FF09FF89307050097
:100F88006FF01FFF03A60500938747009385450070
:100F980023AEC7FEE3E8D7FEE3EAE7F46780000084
:100FA8003367B5009303F0FF13773700631007101A
:100FB800B7877F7F9387F7F70326050083A6050089
:100FC800B372F6003363F600B382F200B3E2620054
:100FD800639272106316D6080326450083A645005F
:100FE800B372F6003363F600B382F200B3E2620034
:100FF800639E720C6316D6060326850083A68500B9
:10100800B372F6003363F600B382F200B3E2620013
:101018006398720C6316D6040326C50083A6C50020
:10102800B372F6003363F600B382F200B3E26200F3
:101038006392720C6316D6020326050183A6050186
:10104800B372F6003363F600B382F200B3E26200D3
:10105800639C720A1305450193854501E30ED6F496
:101068001317060193970601631EF700135706012D
:1010780093D706013305F7409375F50F6390050282
:10108800678000001357070193D707013305F7401E
:101098009375F50F63940500678000001377F70FC9
:1010A80093F7F70F3305F740678000000346050004
:1010B80083C6050013051500938515006314D60033
:1010C800E31606FE3305D640678000001305450089
:1010D80093854500E31CD6FC1305000067800000DB
:1010E8001305850093858500E312D6FC13050000DF
:1010F800678000001305C5009385C500E318D6FA7C
:10110800130500006780000013050501938505019C
:10111800E31ED6F81305000067800000130101FBE9
:1011280023248104232C41033704100013DA4501DA
:1011380023202105232E3103232A5103232481034D
:101148001304F4FF232611042322910423286103A6
:1011580023267103232291032320A103232EB10107
:10116800137AFA7F13090500130C0600938A060008
:101178003374B40093D9F50163060A0A9307F07F24
:101188006304FA1013143400B70780003364F400C2
:10119800135BD501336B8B0093143500130A1AC007
:1011A800930B000013D54A01370910001309F9FF02
:1011B8001375F57F3379590193050C0093DAFA0119
:1011C800630205109307F07F6302F5163704800069
:1011D80013193900336989001354DC01336424017D
:1011E80093153C00130515C09307000013972B00B7
:1011F8003367F7001307F7FF9306E00033C9590177
:10120800330AAA4063E0E616972600009386C64D87
:10121800131727003307D700032707003307D70022
:1012280067000700336BA400630E0B066300040419
:1012380013050400EF109067930755FF1307C001CB
:10124800634CF702130BD001930485FF330BFB406B
:1012580033149400335B6901336B8B00B31499002A
:10126800130AD0C0330AAA406FF09FF3EF1010643E
:10127800130505026FF05FFC130485FD331B89001D
:10128800930400006FF0DFFD336BA40063040B02CE
:1012980093040500130B0400130AF07F930B30002E
:1012A8006FF05FF093040000130A0000930B100026
:1012B8006FF05FEF93040000130AF07F930B200098
:1012C8006FF05FEE33648901630E0406630009045E
:1012D80013050900EF10905D930755FF1307C00130
:1012E800634EF7021304D001930585FF3304F440DD
:1012F8003319B90033548C0033642401B315BC008E
:101308001307D0C03305A7406FF01FEE13050C007C
:10131800EF10D059130505026FF01FFC130485FD6B
:1013280033148C00930500006FF09FFD336489012E
:1013380063020402130409001305F07F93073000C9
:101348006FF0DFEA93050000130500009307100013
:101358006FF0DFE9930500001305F07F9307200085
:101368006FF0DFE86366640163128B4863E0B4489A
:101378009316FB0113D71400139CF401135B1B0095
:10138800B3E4E6001314840093DC8501B3EC8C000D
:1013980093DA0C0193970C0193D70701139D8500ED
:1013A80013050B0093850A002322F100EF10504526
:1013B80093050500930B050013950C0113550501C2
:1013C800EF1050411304050093850A0013050B0024
:1013D800EF1090471315050113D704013365A700D3
:1013E80093890B00637E8500330595019389FBFF84
:1013F80063689501637685009389EBFF3305950152
:101408003304854093850A0013050400EF10503F0C
:1014180093050500930B050013950C011355050161
:10142800EF10503B130B050093850A0013050400C9
:10143800EF109041939D04011315050193DD0D01F3
:10144800B3EDAD0013870B0063FE6D01B38D9D01F5
:101458001387FBFF63E89D0163F66D011387EBFFBC
:10146800B38D9D0193960901B7040100B3E6E60028
:10147800B38D6D41138BF4FF33F76601337B6D0138
:101488001305070093050B0013D406012326D1008A
:101498002324E100EF1010342322A10093050B0050
:1014A80013050400EF101033935B0D019309050039
:1014B80093850B0013050400EF10D031032781003A
:1014C8001304050013850B0093050700EF109030F7
:1014D80003264100330535018326C1001357060151
:1014E8003307A700637437013304940037050100FC
:1014F8001305F5FF93540701B379A70093990901E0
:101508003376A600B3848400B389C90063E89D00DC
:101518001384060063949D0463723C05330CAC018C
:101528003337AC0133079701B38DED001384F6FF11
:1015380063E6BC016394BC036362AC0363E69D008D
:10154800639EB401637C3C01330CAC013337AC01BE
:10155800330797011384E6FFB38DED00B3093C41CF
:10156800B3849D40B3373C01B384F4409305F0FF46
:1015780063889C1A93850A0013850400EF1050288D
:10158800930505002324A10013950C0113550501AB
:10159800EF1050242322A10093850A00138504002C
:1015A800EF10902A832681000327410013150501B7
:1015B80093D7090133E5A700938D0600637EE50004
:1015C80033059501938DF6FF636895016376E50011
:1015D800938DE6FF33059501B304E54093850A0032
:1015E80013850400EF10D021930505002322A100E4
:1015F80013950C0113550501EF10D01D130C0500B0
:1016080093850A0013850400EF10102493990901AB
:10161800032741001315050193D9090133E5A900F2
:1016280093070700637E8501330595019307F7FF4C
:1016380063689501637685019307E7FF3305950194
:1016480093940D01B3E4F4009397040193D7070131
:1016580093050B00B3098541138507002322F10088
:1016680093DD0401EF10101793050B00930A050092
:1016780013850D00EF101016130C050093850D004F
:1016880013850B00EF10101583274100130B05007D
:1016980013850B0093850700EF10D01333058501E0
:1016A80093D70A013385A70063768501B707010040
:1016B800330BFB00B70601009386F6FF935705012D
:1016C8003377D50013170701B3FADA00B387670138
:1016D8003307570163E8F900938504006390F90420
:1016E8006300070433853C019385F4FF6364950325
:1016F8006366F5006314F5026370ED0293161D002E
:1017080033BDA601B30C9D019385E4FF3305950114
:10171800138D06006314F5006304A70193E5150013
:101728001307FA3F6352E01293F7750063800702CC
:1017380093F7F50093064000638AD7009386450027
:10174800B3B5B6003304B40093850600931774004C
:1017580063DA0700B70700FF9387F7FF3374F400D5
:1017680013070A409307E07F63C2E71A9317D4016F
:1017780093D53500B3E7B70013543400B70610000B
:101788009386F6FF3374D400B70610801377F77F7B
:101798009386F6FF131747013374D4001319F90120
:1017A8003364E400336724018320C10403248104E3
:1017B80083244104032901048329C103032A8103E3
:1017C800832A4103032B0103832BC102032C8102CB
:1017D800832C4102032D0102832DC10113850700CB
:1017E800930507001301010567800000130AFAFF3B
:1017F800130C00006FF01FB91389090013040B00C4
:101808009385040093870B00130720006380E7107B
:10181800130730006382E70E13071000E392E7F026
:1018280013040000930700006F00400913890A00A1
:101838006FF09FFD370408009305000013090000AE
:10184800930730006FF05FFC93061000B386E64004
:1018580093078003E3C6D7FC9307F00163C4D70658
:10186800130AEA41B317440133D7D500339A450127
:10187800B3E7E700333A4001B3E747013354D400F4
:1018880013F777006300070213F7F7009306400089
:10189800630AD70013874700B337F7003304F4000F
:1018A8009307070013178400634A07061317D40128
:1018B80093D73700B367F7001354340013070000B9
:1018C8006FF0DFEB930710FEB387E74013070002C2
:1018D800B357F400130500006386E600130AEA43D1
:1018E80033154401336AB500333A4001B3E7470181
:1018F800130400006FF0DFF83704080093070000B6
:101908001307F07F130900006FF05FE7130400006E
:10191800930700001307F07F6FF05FE613040000E1
:1019280093070000130710006FF05FE5130101FA39
:10193800232C8104232631053704100093D945014F
:10194800232A910423206105232E7103232C81036C
:101958001304F4FF232E1104232821052324410511
:1019680023225105232A91032328A1032326B10307
:1019780093F9F97F93040500930B0600138C060076
:101988003374B40013DBF5016388090A9307F07F09
:101998006386F91037098000131434003364240176
:1019A8001359D50133698900131D3500938919C06E
:1019B800930C000013554C01370A1000130AFAFF64
:1019C8001375F57F337A8A0193840B00135CFC014D
:1019D800630405109307F07F6304F516370480004D
:1019E800131A3A00336A8A0013D4DB0133644401C2
:1019F80093943B00130515C09307000013972C0020
:101A08003367F700B389A9001307F7FF9306E000CF
:101A1800B34B8B01938A190063E0E6169726000002
:101A2800938646D0131727003307D70003270700EC
:101A38003307D700670007003369A400630E09065F
:101A48006300040413050400EF104066930755FF74
:101A58001307C001634CF7021309D001130D85FF6A
:101A68003309F9403314A40133D9240133698900B7
:101A7800339DA4019309D0C0B389A9406FF05FF3E7
:101A8800EF10C062130505026FF05FFC130985FDB6
:101A980033992401130D00006FF0DFFD3369A400B2
:101AA80063040902130D0500130904009309F07F6C
:101AB800930C30006FF01FF0130D00009309000025
:101AC800930C10006FF01FEF130D00009309F07FC7
:101AD800930C20006FF01FEE33647A01630E040646
:101AE80063000A0413050A00EF10405C930755FFD2
:101AF8001307C001634EF7021304D001930485FF56
:101B08003304F440331A9A0033D48B00336444010D
:101B1800B3949B009307D0C03385A7406FF0DFEDE7
:101B280013850B00EF108058130505026FF01FFC9A
:101B3800130485FD33948B00930400006FF09FFD20
:101B480033647A016302040213040A001305F07F68
:101B5800930730006FF09FEA93040000130500001C
:101B6800930710006FF09FE9930400001305F07FBE
:101B7800930720006FF09FE837070100130AF7FF6B
:101B8800135C0D0193DD0401337D4D01B3F4440171
:101B980093050D00138504002328E100EF1080430E
:101BA800930C05009385040013050C00EF10804288
:101BB8002326A10093850D0013050C00EF1080412A
:101BC800130B050093050D0013850D00EF108040E1
:101BD8008326C10093D70C013305D5003385A700B0
:101BE8006376D50003270101330BEB0093560501FB
:101BF80033754501B3FC4C0113150501B307950175
:101C0800935C04013374440193050D00130504002B
:101C1800232AD1002326F100EF10C03B2328A1007E
:101C28009305040013050C00EF10C03A130A0500D1
:101C380093850C0013050C00EF10C039130C050038
:101C480093050D0013850C00EF10C0380327010120
:101C58003305450183264101935707013385A700C2
:101C680063764501B7070100330CFC003706010015
:101C780093570501338C87019307F6FF337AF500F4
:101C88003377F700131A0A01135D0901330AEA00D2
:101C98003379F90033874601930509001385040059
:101CA8002328E100232EC100EF10C03293850400E1
:101CB800232CA10013050D00EF10C031232AA10029
:101CC80093050D0013850D00EF10C0309304050037
:101CD8009305090013850D00EF10C02F83264101DD
:101CE800032781013305D500935707013385A700E2
:101CF8006376D5000326C101B384C400B70601008A
:101D08009387F6FF935D0501B3849D00B37DF500CD
:101D18003377F7009305090013050400939D0D011F
:101D2800B38DED00232CD100EF10C02A93050400D9
:101D3800232AA10013050D00EF10C02993050D00FB
:101D48001304050013850C00EF10C028130D0500BF
:101D58009305090013850C00EF10C02703274101E4
:101D680033058500935707013385A70063768500FF
:101D780083268101330DDD0083270101B7060100A9
:101D88009386F6FF330BFB00B377D5003377D70084
:101D980093970701B387E700333A4B01B38787016D
:101DA80033844701330BBB0133079400B33DBB01B8
:101DB800B306B70133BC8701333444019357050197
:101DC8003337970033648C00B3BDB6013304F40095
:101DD800B36DB7013304B4013304A40193D776017A
:101DE800131494003364F4008327C10093149B00F8
:101DF800135B7B01B3E4F400B3349000939796002F
:101E0800B3E46401B3E4F4009317740063D20712D7
:101E180093D7140093F41400B3E497009317F401D4
:101E2800B3E4F400135414001387FA3F6356E01028
:101E380093F774006380070293F7F4009306400059
:101E4800638AD70093874400B3B49700330494009F
:101E5800938407009317740063DA0700B70700FF3D
:101E68009387F7FF3374F40013870A409307E07FE2
:101E780063C6E71893DA34009314D401B3E4540129
:101E880013543400B70710009387F7FF3374F40036
:101E98009377F77F370710801307F7FF939747016A
:101EA8003374E400939BFB013364F400B36774015B
:101EB8008320C10503248105138504000329010536
:101EC800832441058329C104032A8104832A410408
:101ED800032B0104832BC103032C8103832C4103AF
:101EE800032D0103832DC102938507001301010609
:101EF80067800000930B0B001304090093040D0086
:101F080093870C0013072000638AE70E130730003D
:101F1800638CE70C13071000E398E7F01304000044
:101F2800930400006F008008930B0C006FF09FFD76
:101F3800938A09006FF05FEF93061000B386E640BE
:101F480093078003E3CCD7FC9307F00163C4D7065B
:101F5800938AEA41B317540133D7D400B394540198
:101F6800B3E7E700B3349000B3E497003354D400E8
:101F780093F774006380070293F7F4001307400097
:101F8800638AE70093874400B3B49700330494004E
:101F9800938407009317840063CA07069317D40134
:101FA80093D43400B3E497001354340013070000AB
:101FB8006FF05FED930710FEB387E740130600024A
:101FC800B357F400130700006386C600938AEA43F8
:101FD80033175401B3649700B3349000B3E4970007
:101FE800130400006FF0DFF83704080093040000C2
:101FF8001307F07F930B00006FF0DFE81304000075
:10200800930400001307F07F6FF0DFE7130400006C
:1020180093040000130710006FF0DFE6130101FDC1
:1020280023229102232A510193547501B70A800093
:102038002320210323286101938AFAFF2326110212
:1020480023248102232E3101232C410123267101EF
:102058002324810193F4F40F138B0500B3FAAA002B
:102068001359F501638804089307F00F6384F40A91
:10207800939A3A00B7070004B3EAFA00938414F875
:10208800930B000013557B01370480001304F4FF01
:102098001375F50F33746401135BFB01630C0508BA
:1020A8009307F00F6308F50A13143400B707000408
:1020B8003364F400130515F89307000013972B00F9
:1020C8003367F7001307F7FF9306E000B349690188
:1020D800338AA44063E0E60A9716000093864668B0
:1020E800131727003307D700032707003307D70044
:1020F80067000700638A0A0213850A00EF00107B55
:102108009307B5FF9304A0F8B39AFA00B384A440E8
:102118006FF01FF79304F00F930B2000E3840AF687
:10212800930B30006FF01FF693040000930B100020
:102138006FF05FF5630A040213050400EF001077DF
:102148009307B5FF3314F4009307A0F83385A7402D
:102158006FF09FF61305F00F93072000E30004F6D5
:10216800930730006FF09FF51305000093071000E8
:102178006FF0DFF4131B540063F68A12130AFAFF98
:1021880013090000935B0B013704010093850B00D2
:102198001304F4FF13850A00EF00906633748B0074
:1021A80093050500130C050013050400EF00906269
:1021B8009304050093850B0013850A00EF00D0688F
:1021C80013590901131505013365A90013090C00FA
:1021D800637E9500330565011309FCFF636865019B
:1021E800637695001309ECFF33056501B304954048
:1021F80093850B0013850400EF009060930505009C
:10220800130C050013050400EF00D05C930A0500C9
:1022180093850B0013850400EF0010631315050167
:1022280013040C00637E5501330565011304FCFF9C
:1022380063686501637655011304ECFF3305650196
:102248001319090133055541336989003335A00055
:102258003364A9001307FA076350E00A9377740000
:10226800638A07009377F400930640006384D700DD
:10227800130444009317440063DA0700B70700F813
:102288009387F7FF3374F40013070A089307E00FE6
:102298001354340063D2E70C130400001307F00F43
:1022A8006F00800B1399FA0193DA1A006FF09FED13
:1022B8009309090013840A0093870B001307200071
:1022C800E38CE7FC130730006382E708130710006C
:1022D800E392E7F813040000130700006F00C0073B
:1022E80093090B006FF09FFD37044000930900002D
:1022F800930730006FF09FFC93071000B387E74007
:102308001307B001E348F7FC1305EA09B357F400D3
:102318003314A4003334800033E4870093777400C7
:10232800638A07009377F400130740006384E7008B
:10233800130444009317540013543400E3DE07F8E1
:1023480013040000130710006F0000013704400059
:102358001307F00F93090000370580001305F5FFF8
:102368003374A400370580801305F5FF1377F70F42
:102378003374A400131777011395F9013364E4004B
:102388003365A4008320C10203248102832441020F
:10239800032901028329C101032A8101832A4101FA
:1023A800032B0101832BC100032C810013010103BE
:1023B80067800000130101FD2322910223202103DD
:1023C800B704800013597501232E310123267101AA
:1023D8009384F4FF2326110223248102232C410134
:1023E800232A5101232861012324810123229101F9
:1023F8001379F90F938B0500B3F4A4009359F501F1
:10240800630A09089307F00F6306F90A93943400E6
:10241800B7070004B3E4F400130919F8130B00001C
:1024280013D57B01370480001304F4FF1375F50FEF
:102438003374740193DBFB01630E05089307F00FF7
:10244800630AF50A13143400B70700043364F40070
:10245800130515F89306000093172B00B3E7D70070
:102468003309A9009387F7FF1307E00033CA7901FE
:10247800930A19006360F70A171700001307073259
:1024880093972700B387E70083A70700B387E70080
:1024980067800700638A040213850400EF00104177
:1024A8009307B5FF1309A0F8B394F4003309A940C2
:1024B8006FF0DFF61309F00F130B2000E38204F628
:1024C800130B30006FF0DFF513090000130B100039
:1024D8006FF01FF5630A040213050400EF00103DB6
:1024E8009307B5FF3314F4009307A0F83385A7408A
:1024F8006FF05FF61305F00F93062000E30E04F467
:10250800930630006FF05FF5130500009306100086
:102518006FF09FF4370C0100130BFCFF93DB0401F1
:10252800935C0401B3F464013374640193050400FB
:1025380013850400EF00102A930504009309050091
:1025480013850B00EF0010291304050093850C0078
:1025580013850B00EF001028930B050093850400EA
:1025680013850C00EF0010273305850093D7090168
:102578003385A70063748500B38B8B01B37765013E
:1025880093970701B3F96901B3873701139467007B
:102598003334800093D7A70113550501B367F400BE
:1025A80033047501131464003364F4009317440072
:1025B80063D6070E935714001374140033E487008E
:1025C8001387FA076350E00E93777400638A070055
:1025D8009377F400930640006384D7001304440003
:1025E8009317440063DA0700B70700F89387F7FFEB
:1025F8003374F40013870A089307E00F63C4E710E5
:10260800935734006F000003138A090013840400F1
:1026180093060B00930720006386F60E930730009D
:10262800638AF60C130610009307000013070000D6
:10263800E398C6F8370480001304F4FF3705808058
:10264800B3F787001305F5FF8320C1020324810235
:102658001377F70FB3F7A700131777011315FA01CC
:10266800B3E7E70083244102032901028329C1015A
:10267800032A8101832A4101032B0101832BC10015
:10268800032C8100832C410033E5A70013010103CB
:1026980067800000138A0B006FF0DFF7930A0900C8
:1026A8006FF01FF293071000B387E7401307B001DC
:1026B8006340F706938AEA09B357F40033145401C8
:1026C8003334800033E4870093777400638A07000B
:1026D8009377F400130740006384E7001304440071
:1026E8009317540063CA0702935734001307000076
:1026F8006FF05FF4B70740001307F00F130A0000EC
:102708006FF05FF3930700001307F00F6FF09FF26D
:10271800930700006FF09FFD930700001307100058
:102728006FF05FF1B70780009387F7FF130101FF90
:1027380033F7A7009356750113D67501B3F7B700A1
:10274800232291002320210193F6F60F1318370056
:102758001376F60F23261100232481001307F00FA8
:102768009354F501138906001305060093D5F50166
:10277800939737006314E6006394070093C5150028
:102788003387C640639A951A6356E00A63160606AD
:10279800639C07009307F00F638CF6049307080007
:1027A800138506006F00C0141307F7FF631E0702A6
:1027B800B38707011385060013975700635A07125A
:1027C800130515001307F00F630EE5323707007E77
:1027D80093F617001307F7FF93D71700B3F7E7002F
:1027E800B3E7D7006F00C0101306F00F639EC60052
:1027F800930708006F0040071306F00FE38AC6FE30
:1028080037060004B3E7C7001306B0016356E600B5
:10281800930710006FF0DFF9130600023306E64055
:10282800B3D5E700B397C700B337F000B3E7F500B7
:102838006FF01FF863000708639C0602631808001E
:102848001307F00F6316E60A6F0000029306F0FF05
:102858006316D700B38707016FF01FF69306F00FD2
:102868001347F7FF6310D6021305F00F6F004008F7
:102878009306F00FE30AD6FEB70600043307E040DC
:102888003368D8009306B00163D6E600130710003A
:102898006F00C001930600023356E8003387E64014
:1028A8003317E8003337E0003367E600B387E70003
:1028B8006FF09FF0138516001376F50F13071000BD
:1028C8006342C70663940604130500006302080206
:1028D80063860722B387070113975700635A0700D7
:1028E800370700FC1307F7FFB3F7E70013051000DD
:1028F80013F77700630A072013F7F70093064000E1
:102908006304D720938747006F000020E30E08F484
:10291800E38007EEB70700021305F00F93040000E9
:102928006F00801E1307F00F630EE51C3307F800D5
:10293800935717006FF0DFFB6350E0086316060437
:10294800E38A07E41307F7FF63140702B307F840A5
:102958001385060013975700E35C07F83704000453
:102968001304F4FF33F48700130905006F00801384
:102978001306F00FE38EC6E61306B0016350E602B5
:10298800930710006FF09FFC1306F00FE382C6E672
:1029980037060004B3E7C7006FF01FFE13060002F6
:1029A800B3D5E7003307E640B397E700B337F00045
:1029B800B3E7F5006FF09FF963020708639E06020C
:1029C800631808001307F00F938405006FF09FE762
:1029D8009306F0FF6318D700B38707419384050077
:1029E8006FF05FF79306F00F1347F7FF6310D602F7
:1029F800938405006FF05FE79306F00FE30AD6FEB5
:102A0800B70600043307E0403368D8009306B001E6
:102A180063D6E600130710006F00C001930600029A
:102A28003356E8003387E6403317E8003337E000D1
:102A38003367E600B387E7406FF05FFA1387160045
:102A48001377F70F130610006344E604639C06022D
:102A58006318080063980712130500006FF01FEC55
:102A6800638607123307F84093165700B387074168
:102A780063CA061093070700631007069307000050
:102A88006FF09FFDE31608E8E39407F66FF09FE800
:102A98003304F84013175400635407043384074180
:102AA8009384050013050400EF0040601305B5FF8B
:102AB8003314A400634A2503330525411305150083
:102AC80013070002B357A4003305A7403314A4002A
:102AD80033348000B3E78700130500006FF05FE12F
:102AE800E30E04F86FF01FFCB70700FC9387F7FFAD
:102AF8003305A940B377F4006FF09FDF9307080010
:102B08006FF01FDF9307000013975700635E0700FD
:102B1800130515001307F00F630EE506370700FCD1
:102B28001307F7FFB3F7E7001307F00F93D7370042
:102B38006318E50063860700B707400093040000A8
:102B4800370780001307F7FF1375F50FB3F7E70092
:102B580013177501370580808320C1000324810085
:102B68001305F5FF33F5A7009394F4013365E500E9
:102B780033659500032901008324410013010101F5
:102B880067800000938405006FF01FF59307080025
:102B98006FF09FF4930700006FF01FF9370680006D
:102BA800135775019307F6FF1377F70F9305E0079F
:102BB800B3F7A7009356F50163F6E5049305D0092A
:102BC80063FAE500370500801345F5FF3385A60055
:102BD8006780000033E5C7009307500963DCE7000E
:102BE8001307A7F63315E500638006023305A040F6
:102BF80067800000930760093387E7403355E50095
:102C08006FF09FFE1305000067800000130101FFAD
:102C1800232611002324810023229100630205103A
:102C2800130405009354F501635405003304A040D0
:102C380013050400EF0080479307E009B387A74016
:102C4800130760096340F706130780006356A7005F
:102C5800130585FF3314A400370580001305F5FF1D
:102C680093F7F70F3374A40013957701B7078080A3
:102C78009387F7FF3374F400B70700803364A40028
:102C880093C7F7FF1395F4013374F4003365A40078
:102C98008320C10003248100832441001301010122
:102CA80067800000130790096350F702130750006C
:102CB8003307A7409306B5013357E4003314D40013
:102CC8003334800033648700130750006356A7002D
:102CD8001307B5FF3314E400370700FC1307F7FFA9
:102CE800937674003377E400638A06001374F40063
:102CF800930640006304D400130747009316570057
:102D080063DC0600B70700FC9387F7FF3377F7000B
:102D18009307F009B387A740135437006FF0DFF328
:102D28001304000093070000930400006FF0DFF223
:102D380093577501130101FF93F7F70F23248100BF
:102D48001387170037048000232291001304F4FF2F
:102D5800232611001377F70F930610003374A4008D
:102D68009354F50163D2E606138507389357340068
:102D78001314D401370710001307F7FFB3F7E70060
:102D8800370710801307F7FF1375F57F13154501F3
:102D9800B3F7E70037070080B3E7A7001347F7FF4B
:102DA8001395F401B3F7E70033E7A7008320C100C8
:102DB80013050400032481008324410093050700C0
:102DC800130101016780000063940704630204068D
:102DD80013050400EF00802D9307A00063C2A7022B
:102DE8009307B000B387A74013075501B357F40002
:102DF8003314E400130790383305A7406FF09FF7AA
:102E0800930755FFB317F400130400006FF09FFEFB
:102E180093070000630A040093573400370708003B
:102E28001314D401B3E7E7001305F07F6FF09FF4A4
:102E380093070000130500006FF0DFF3370610005A
:102E48001306F6FF3376B60013D845019357D5011C
:102E58001378F87F1316360033E6C7009307180077
:102E680093F7F77F9306100093D5F50113173500F4
:102E780063D6F60A930608C89307E00F63C2D70C17
:102E88006340D008930790FE63C4F612B70780002A
:102E98001305E0013366F6003305D5409307F001CA
:102EA80063C8A702130828C8B3170701B337F0008F
:102EB800331606013355A700B3E7C700B367F5001B
:102EC8009306000013F77700630007086F00C00E31
:102ED8009307E0FFB386D74093070002B356D600A6
:102EE800930800006306F500130828CAB318060102
:102EF800B3E7E800B337F000B3E7F6006FF05FFC24
:102F0800131565003335A000131636009357D70103
:102F18003366C500B367F6006FF0DFFAB367E60003
:102F280063160800B337F0006FF09FF99306F00FAF
:102F3800638C070013163600B70700026FF09FFD79
:102F4800930700009306F00F13975700635E07007E
:102F5800938616001307F00F638AE606370700FC0E
:102F68001307F7FFB3F7E7001307F00F93D73700FE
:102F78006398E60063860700B707400093050000E2
:102F8800370580001305F5FFB3F7A70037058080E4
:102F98001305F5FF93F6F60F93967601B3F7A7009E
:102FA8009395F501B3E7D70033E5B70067800000D4
:102FB800930710009306000013F7F700130640006C
:102FC800E304C7F8938747006FF01FF893070000E2
:102FD8006FF09FF9130605001305000093F615001E
:102FE800638406003305C50093D515001316160033
:102FF800E39605FE678000006340050663C6050684
:1030080013860500930505001305F0FF630C0602FF
:1030180093061000637AB6006358C00013161600B2
:1030280093961600E36AB6FE1305000063E6C50032
:10303800B385C5403365D50093D6160013561600E0
:10304800E39606FE6780000093820000EFF05FFBC6
:1030580013850500678002003305A04063D805008A
:10306800B305B0406FF0DFF9B305B04093820000BC
:10307800EFF01FF93305A04067800200938200003B
:1030880063CA0500634C0500EFF09FF71385050040
:1030980067800200B305B040E35805FE3305A04041
:1030A800EFF01FF63305B04067800200B707010054
:1030B800637AF5029307F00FB3B7A7009397370029
:1030C800130700023307F740B357F5001705000050
:1030D80013058570B307F50003C507003305A7403E
:1030E800678000003707000193070001E36AE5FCE9
:0830F800930780016FF0DFFC7B
:10310000130101FF23261100EFD00F9F8320C10080
:10311000B70710F023A007F2130500001301010107
:0431200067800000C4
:103124004448525953544F4E452050524F475241F0
:103134004D2C20534F4D4520535452494E470000C7
:103144004468727973746F6E652042656E63686D4E
:1031540061726B2C2056657273696F6E20322E314A
:1031640020284C616E67756167653A204329000029
:1031740050726F6772616D20636F6D70696C656406
:10318400207769746820277265676973746572278C
:1031940020617474726962757465000050726F679F
:1031A40072616D20636F6D70696C656420776974FA
:1031B400686F757420277265676973746572272058
:1031C400617474726962757465000000506C6561A5
:1031D4007365206769766520746865206E756D6215
:1031E4006572206F662072756E73207468726F75D5
:1031F4006768207468652062656E63686D61726BD0
:103204003A200000457865637574696F6E207374A5
:10321400617274732C2025642072756E7320746837
:10322400726F756768204468727973746F6E650A8B
:1032340000000000457865637574696F6E20656EE3
:103244006473000046696E616C2076616C75657309
:10325400206F6620746865207661726961626C65AE
:1032640073207573656420696E20746865206265D7
:103274006E63686D61726B3A00000000496E745FA2
:10328400476C6F623A20202020202020202020201C
:103294002025640A00000000202020202020202077
:1032A40073686F756C642062653A20202025640A77
:1032B40000000000426F6F6C5F476C6F623A202021
:1032C40020202020202020202025640A0000000047
:1032D40043685F315F476C6F623A202020202020D2
:1032E400202020202025630A000000002020202028
:1032F4002020202073686F756C642062653A20205A
:103304002025630A0000000043685F325F476C6F4A
:10331400623A202020202020202020202025630A1B
:10332400000000004172725F315F476C6F625B386E
:103334005D3A2020202020202025640A000000007F
:103344004172725F325F476C6F625B385D5B375D01
:103354003A2020202025640A00000000202020209C
:103364002020202073686F756C642062653A2020E9
:10337400204E756D6265725F4F665F52756E732085
:103384002B203130000000005074725F476C6F6274
:103394002D3E000020205074725F436F6D703A2000
:1033A40020202020202020202025640A0000000066
:1033B400202020202020202073686F756C642062F8
:1033C400653A20202028696D706C656D656E7461A6
:1033D40074696F6E2D646570656E64656E74290022
:1033E400202044697363723A20202020202020206A
:1033F400202020202025640A000000002020456EA3
:10340400756D5F436F6D703A2020202020202020AE
:103414002025640A000000002020496E745F436F79
:103424006D703A2020202020202020202025640AAE
:103434000000000020205374725F436F6D703A20C7
:1034440020202020202020202025730A00000000B6
:10345400202020202020202073686F756C64206257
:10346400653A2020204448525953544F4E45205029
:10347400524F4752414D2C20534F4D4520535452E7
:10348400494E47004E6578745F5074725F476C6FA5
:10349400622D3E00202020202020202073686F759C
:1034A4006C642062653A20202028696D706C656D1B
:1034B400656E746174696F6E2D646570656E6465A4
:1034C4006E74292C2073616D652061732061626FB5
:1034D40076650000496E745F315F4C6F633A20205B
:1034E40020202020202020202025640A0000000025
:1034F400496E745F325F4C6F633A20202020202095
:10350400202020202025640A00000000496E745FFA
:10351400335F4C6F633A202020202020202020207D
:103524002025640A00000000456E756D5F4C6F63D2
:103534003A20202020202020202020202025640A3A
:10354400000000005374725F315F4C6F633A2020B7
:1035540020202020202020202025730A00000000A5
:10356400202020202020202073686F756C64206246
:10357400653A2020204448525953544F4E45205018
:10358400524F4752414D2C2031275354205354520B
:10359400494E47005374725F325F4C6F633A202088
:1035A40020202020202020202025730A0000000055
:1035B400202020202020202073686F756C642062F6
:1035C400653A2020204448525953544F4E452050C8
:1035D400524F4752414D2C2032274E4420535452CF
:1035E400494E47004D656173757265642074696D59
:1035F4006520746F6F20736D616C6C20746F206F25
:10360400627461696E206D65616E696E6766756C62
:1036140020726573756C747300000000506C6561F2
:10362400736520696E637265617365206E756D6282
:103634006572206F662072756E730000436C6F6351
:103644006B206379636C65733D2564200A00000078
:10365400444D49505320706572204D687A3A2020B9
:103664002020202020202020202020202020202056
:1036740020202020202020202020202000000000C6
:1036840025642E00256400004448525953544F4E7B
:10369400452050524F4752414D2C2031275354203E
:1036A400535452494E4700004448525953544F4EC4
:1036B400452050524F4752414D2C2032274E442032
:1036C400535452494E4700004448525953544F4EA4
:1036D400452050524F4752414D2C2033275244200D
:1036E400535452494E47000028E2FFFF3CE1FFFFDC
:1036F40048E1FFFF3CE1FFFF14E2FFFF3CE1FFFF75
:1037040048E1FFFF28E2FFFF28E2FFFF14E2FFFF8A
:1037140048E1FFFF14E1FFFF14E1FFFF14E1FFFFA5
:1037240050E1FFFFE4E7FFFFE4E7FFFF08E8FFFFE6
:10373400D8E7FFFFD8E7FFFFC8E8FFFF08E8FFFF6F
:10374400D8E7FFFFC8E8FFFFD8E7FFFF08E8FFFF5F
:10375400D4E7FFFFD4E7FFFFD4E7FFFFC8E8FFFF8C
:103764003CEBFFFF78EBFFFF84EBFFFF78EBFFFF01
:10377400F0EBFFFF78EBFFFF84EBFFFF3CEBFFFF79
:103784003CEBFFFFF0EBFFFF84EBFFFF54EBFFFF8D
:1037940054EBFFFF54EBFFFF8CEBFFFF7CEEFFFFCE
:1037A4007CEEFFFFFCEEFFFF74EEFFFF74EEFFFF05
:1037B4005CEFFFFFFCEEFFFF74EEFFFF5CEFFFFF2B
:1037C40074EEFFFFFCEEFFFF70EEFFFF70EEFFFFF5
:1037D40070EEFFFF5CEFFFFF00010202030303032F
:1037E400040404040404040405050505050505058D
:1037F400050505050505050506060606060606066D
:103804000606060606060606060606060606060654
:10381400060606060606060607070707070707073C
:103824000707070707070707070707070707070724
:103834000707070707070707070707070707070714
:103844000707070707070707070707070707070704
:1038540007070707070707070808080808080808EC
:1038640008080808080808080808080808080808D4
:1038740008080808080808080808080808080808C4
:1038840008080808080808080808080808080808B4
:1038940008080808080808080808080808080808A4
:1038A4000808080808080808080808080808080894
:1038B4000808080808080808080808080808080884
:1038C4000808080808080808080808080808080874
:0838D4000808080808080808AC
:1038E0000000000080842E41000000205FA01242F2
:0C38F000F90295503353DE470000C84237
:040000058000000077
:00000001FF
